:020000040000FA
:02000000902945
:08000800A4000308AD008B0108
:10001000C00B1128D230C000C10B1128C20A043015
:10002000C1003520B8013718381438088600851DFE
:100030003120422003111108193C031D2820031907
:100040002C20003081002D08830024088B16090025
:10005000910A9A0A900A0800143091009A009001BF
:100060000800B00A1008B1000800031142083C3C27
:10007000031D0800C201C30B08001930BB00043087
:100080007723080010086E2085001A0884000008F5
:100090004F20B80037183814380886000800820747
:1000A00000349034EC34F834B2347A347E349834FA
:1000B000FE34FA34DE34203401346634AA34643435
:1000C0006E344634743434342E34D634AE344E3434
:1000D00098340E349A348E34F434F4348207013474
:1000E0000434003403340534023482070A34013402
:1000F0000134023402340334033404340434053448
:100100000534063406340734073408340834093417
:1001100009341A341A3411341134123412341334A9
:100120001334143414341534153416341634173487
:10013000173418341834193419342A342A34213431
:1001400021342234223423342334243424342534F7
:1001500025342634263427342734283428342934C7
:1001600029343A343A343134313432343234333459
:100170003334343434343534353436343634373437
:10018000373438343834393439344A344A344134E1
:1001900041344234423443344334443444344534A7
:1001A0004534463446344734473448344834493477
:1001B00049345A345A345134513452345234533409
:1001C00053345434543455345534563456345734E7
:1001D000573458345834593459346A346A34613491
:1001E0006134623462346334633464346434653457
:1001F0006534663466346734673468346834693427
:1002000069347A347A3471347134723472347334B8
:100210007334743474347534753476347634773496
:10022000773478347834793479348A348A34813440
:100230008134823482348334833484348434853406
:1002400085348634863487348734883488348934D6
:1002500089349A349A34BB34BB34BB34BB34BB349A
:10026000BB34BB34BB34BB34BB34BB34BB34BB3416
:100270003A343A342934293428342834273427347A
:1002800026342634253425342434243423342334AA
:1002900022342234213421342A342A3419341934B2
:1002A00018341834173417341634163415341534FA
:1002B000143414341334133412341234113411340A
:1002C0001A341A340934093408340834073407342A
:1002D000063406340534053404340434033403345A
:0C02E00002340234013401340A3482027A
:100320008316183085000030860083128316513002
:10033000810083120030810014309A0091009001F6
:10034000940195019601970198019901B0018F23BD
:10035000B701AA298B168B17B121F521C222C22120
:10036000AA29043087230311193C031D080000301B
:1003700094009500990010309600133097001C30BF
:100380009800B729340835020318D029C729350841
:100390002C02031CE72934082C020318D929080071
:1003A00035082C020318E72934082C02031CD9292C
:1003B00008003718080037140030940095009800A2
:1003C00099000A309600133097006A230800371C02
:1003D0000800371000309400950099000A3096000C
:1003E0001430970098006A23080003113008643C19
:1003F000031D080005309400103095000D30960064
:10040000153097001630980000309900B001822214
:1004100003113108013C0319080003113108023CA3
:100420000319582203113108033C03191822FA2931
:1004300005309400103095000D3096000A3097007A
:100440001430980014309900822203113108013CC5
:10045000031908003108023C0319422A3108033C01
:1004600003194D2A0A309400143095001430960078
:1004700000309700350875209F2233089800320815
:100480009900242A03113508003C0319322AB503C8
:100490003508BB0012307723322A03113508A03CFF
:1004A0000319322AB50A3508BB0012307723322AE5
:1004B00005309400103095000D3096000030970004
:1004C0000A30980013309900822203113108013C50
:1004D000031908003108023C0319892A3108033C3A
:1004E0000319942A0A3094001330950000309600C6
:1004F00000309700340875209F2233089800320896
:100500009900642A03113008323C031D822AB0018D
:10051000080003113408003C0319722AB40334089C
:10052000BB0011307723722A03113408A03C031951
:10053000722AB40A3408BB0011307723722AB20140
:10054000B3019201A3000310A30C03183216B20CDE
:10055000920A12080311043C031DA32A0310A30CE2
:1005600003183316B30C920A12080311083C031D3A
:10057000AE2AB2133213B2123212B3133313B312C0
:10058000331208000E30970017309800C822080078
:100590004B23013E1D23031D0800CC303323443080
:1005A0003323BE3065231D23CC303323BE303323A9
:1005B0004B23AC004B23AB00DE2208002B080311B9
:1005C000FF3C03190B30031D00309400F422270870
:1005D000950095131513951215122608960096137B
:1005E0001613961216120800A701A6019201031114
:1005F0002B08FF3C031DFE2A0319022B2C08752033
:10060000A300062B2C087521A300062B0310A30CB6
:1006100003182616A60C920A12080311043C031DA7
:10062000062B0310A30C03182716A70C920A120816
:100630000311083C031D112B080005128316051237
:100640008312963065238B138B1B232B8316051681
:1006500083121130652305081039A1004B30652342
:1006600021088B170800A2000830A1008B138B1BF8
:10067000362B051283160512831202306523A20C55
:100680000318051611306523831605168312A10B76
:10069000362B8B1708000830A1008B138B1B4D2BBA
:1006A0000512831605128312023065238316051680
:1006B000831205081039A300FF3EA20C11306523F8
:1006C000A10B4D2B22088B170800A0006400A00B83
:1006D000662B0800FF30A800FF30A9000A30AA00EE
:1006E000A80B702BA90B702BAA0B702B080089008C
:1006F0003B088800831608158B1355308900AA30F3
:10070000890088140811831208088B1708008900D3
:100710008B138316081483128B17080808001130F6
:100720008723B40012308723B500FA30C3003408A1
:10073000A03C031CA0233508A03C031CA3230800F5
:0E0740003230B40008003C30B500080008005C
:02400E00F23F7F
:00000001FF
